:1000000008308A0000280000D3346D38EC32202AF2
:10001000E832F236EF36653AE8327210A0060A008E
:10002000533A613B781DA01258147039EF3165378F
:10003000F430A9060A00D43270366F3A6110753B6D
:10004000EE347439A0346F1DA0124C32A0210D057E
:100050000000CE30F032F434A031EC30EE35751DB6
:10006000A0124C32A03656100D0500015039EF3A5F
:10007000641DA0124C32A03641100D050001CB309A
:10008000F030E334F430203DE23CF4326B1DA0123A
:100090004C32A03641340D050001CB30F030E33452
:1000A000F430A036613C3A1025266410ED20E806B5
:1000B0000A00533A613B3A10252664102838F2377B
:1000C000E3326E3AE1140D050000A01320088316F8
:1000D0008700831287130830F8006E280000F81795
:1000E0007F28F813C40C03188717031C871378178D
:1000F0007F287813F80B72287D28000087173F307F
:100100008400840B81280000F81B7128781B792853
:100110000800831603178C170C14000000008312CC
:100120000C087F390319CD280313BB0003170D08F2
:100130000313BC0003170F080313BD003B08C400E2
:1001400065203C0803178D0003133D0803178F003B
:1001500083168C170C140000000083120C0D0E0D7A
:100160007F390319CD280313BB0003170D080313B0
:10017000BC0003170F080313BD003B08C400652033
:100180003C0803178D0003133D0803178F008D0AE9
:1001900003198F0A03138928031703138A150A12F8
:1001A0006D280830F80000008711A0112008831680
:1001B000870000008312BB0D0712031CE5282016E0
:1001C000200883168700E92883122012200883164E
:1001D000870000008312A015200883168700831271
:1001E000871DF028F80BD32800008711A0112008E4
:1001F00083168700000083122016200883168700CC
:10020000000000008312A0152008831687008312C7
:10021000871D0829F8010000071A78148711A0111A
:1002200020088316870083120712201220088316E5
:100230008700831208000830BC007708BD00201634
:1002400020088316870000008312A015200883165B
:1002500087008312871D2A29071A0314071E03101B
:10026000F80D0000A0112008831687008312871163
:10027000BC0B1F292016200883168700000083125C
:1002800007123D0803194929201220088316870008
:1002900083120000A0152008831687008312871D93
:1002A0004F2900008711A011200883168700000045
:1002B0008312071220122008831687008312080079
:1002C0003C30840083130008031973290230F800BE
:1002D000F701F70B6929F80B68299730F700F70B3E
:1002E0006F29800B66290800831603178C170C14DE
:1002F000000000000318A32983120C087F390313A0
:10030000BC0003170D080313BD0003170F080313E8
:10031000BE003C08C40065203D0803178D00031390
:100320003E0803178F0083168C170C140000000082
:1003300083120313BB0B9D29A02983160317A3293E
:10034000C2298316031783120C0D0E0D7F39031378
:10035000BC0003170D080313BD0003170F08031398
:10036000BE003C08C40065203D0803178D00031340
:100370003E0803178F008D0A03198F0A0310031319
:10038000BB0B74290800BC1BD5290F30F7003B0EAE
:10039000F7050A3077020318D0293030F707D22941
:1003A0003C08F7077708C40065200F30BB050A300A
:1003B0003B020318DD293030DF29BC133C08BB07A2
:1003C0003B08C40065208A150A123729F801F90193
:1003D000F701FA013E08031DF0293D0803190A2A16
:1003E0001030BF000310BB0DBC0DF70DFA0D3E0819
:1003F0007A02031DFD293D087702031C062A3D08E9
:10040000F702031CFA033E08FA020314F80DF90D73
:10041000BF0BF2298A150A12CE2EC3010408C200AE
:100420004310831B4314BC1F1D2AC217421EC20A5D
:10043000BB09BC09BB0A0319BC0A3C0EF038BE005C
:10044000BE07E23EBF00323EC1003C080F39BF0785
:10045000BF07C107E93EC000C007C0073B0E0F3908
:10046000C007C107C00DC10DC109C10D3B080F393F
:10047000C107BE0D0730BD000A30C107C003031C11
:100480003D2AC007BF03031C412ABF07BE03031C4C
:10049000452ABE07BD03031C492A3D30840083134F
:1004A00007304205421384034205031D5E2A421AA7
:1004B000840A421A5E2A2030F7007B2A84074130E2
:1004C0000402031942170008F700031D6F2A421B9C
:1004D0006F2A421A892AC2196F2A20307A2AC21F2B
:1004E000772A2D30F70084034213C2137B2AC215EA
:1004F00042123030F707BC010408BB003C10831BDC
:100500003C147708C40065203B08840083133C1822
:0A0510008317840A421F5F2A0800C7
:10100000840183131F308305713083168F000F080E
:101010008312A01320088316870083128717831674
:1010200003170908C039890003131F129F120030EB
:10103000031788008312870188018901FF30031399
:10104000A000831603170908C039890003131F1273
:101050009F12003003178800831203131F139F137E
:1010600083169F1383121F149412A0122008831654
:101070008700831220162008831687008312A01190
:1010800020088316870001308312940000308316F5
:1010900094000108C739083881008312900100309C
:1010A000F800920000308316920083122015200869
:1010B000831687008312970183169B019C010130E0
:1010C0009D008312031787018801890104308D0078
:1010D00000308F008A11031389288A1520162008F2
:1010E0008316870000008312A0152008831687004E
:1010F00000008312071220122008831687000000C8
:1011000083128711A011200883168700E130831213
:10111000BB008A11D1208A1578083A1078183A1441
:10112000201220088316870000008312A0152008D3
:10113000831687008312871D9B2800009F280000CC
:101140002016200883168700000001308312BA069B
:10115000201620088316870000008312A01520089F
:1011600083168700000083120712201220088316BE
:101170008700000083128711A011200883168700C2
:10118000E0308312BB008A11D1208A158030BB0069
:101190008A11D1208A1520122008831687000000AA
:1011A0008312A0152008831687008312871DD62876
:1011B0000000DA28000020162008831687000000AF
:1011C0008312201620088316870000008312A015C2
:1011D00020088316870000008312071220122008BF
:1011E00083168700000083128711A0112008831640
:1011F0008700E1308312BB008A11D1208A150130AB
:10120000F7008A111B218A157808B90020122008DE
:101210008316870000008312A0152008831687001C
:101220008312871D112900001529000020162008AF
:1012300083168700000004308312BB00FA30BC0024
:101240008A1160218A15BB0B1E29103003178D00EF
:1012500000308F00031007300313BB008A11742184
:101260008A153908BB003730BC008A11C3298A159A
:10127000143003178D0000308F0003140C3003135B
:10128000BB008A1174218A15201620088316870056
:1012900000008312A0152008831687000000831227
:1012A000071220122008831687000000831287117E
:1012B000A011200883168700E0308312BB008A113A
:1012C000D1208A150130BB008A11D1208A15201245
:1012D00020088316870000008312A01520088316BB
:1012E00087008312871D72290000762900002016CE
:1012F000200883168700000083122016200883161A
:10130000870000008312A0152008831687000000C4
:101310008312071220122008831687000000831210
:101320008711A011200883168700AA308312BB0002
:101330008A11D1208A150C30BB008A11D1208A1560
:10134000201620088316870000008312A0152008AD
:101350008316870000008312871DAC290712201214
:10136000200883168700000083128711A01120082F
:1013700083168700AB308312BB008A11D1208A15F7
:10138000F7018A111B218A157808A1002012200874
:101390008316870000008312A0152008831687009B
:1013A0008312871DD1290000D529000020162008AE
:1013B00083168700000083122016200883168700FA
:1013C00000008312A01520088316870000008312F6
:1013D000071220122008831687000000831287114D
:1013E000A011200883168700AA308312BB008A113F
:1013F000D1208A150D30BB008A11D1208A15201604
:1014000020088316870000008312A0152008831689
:10141000870000008312871D0B2A07122012200864
:1014200083168700000083128711A01120088316FD
:101430008700AB308312BB008A11D1208A15F701D7
:101440008A111B218A157808A20020122008831611
:10145000870000008312A0152008831687008312DE
:10146000871D302A0000342A000020162008831629
:1014700087000000831220162008831687000000D2
:101480008312A0152008831687000000831207121C
:101490002012200883168700000083128711A011F4
:1014A000200883168700AA308312BB008A11D1203E
:1014B0008A150830BB008A11D1208A152012200815
:1014C0008316870000008312A0152008831687006A
:1014D0008312871D692A00006D2A0000201620084B
:1014E00083168700000083122016200883168700C9
:1014F00000008312A01520088316870000008312C5
:10150000071220122008831687000000831287111B
:10151000A011200883168700AB308312BB008A110C
:10152000D1208A15F7018A111B218A157808A3009A
:10153000201220088316870000008312A0152008BF
:10154000831687008312871DA32A0000A72A0000A4
:10155000201620088316870000008312201620081A
:101560008316870000008312A015200883168700C9
:101570000000831207122012200883168700000043
:1015800083128711A011200883168700AA308312C6
:10159000BB008A11D1208A150930BB008A11D120E5
:1015A0008A15201220088316870000008312A015D8
:1015B0002008831687008312871DDC2A0000E02A9A
:1015C00000002016200883168700000083122016D2
:1015D00020088316870000008312A01520088316B8
:1015E000870000008312071220122008831687004C
:1015F000000083128711A011200883168700AB30EA
:101600008312BB008A11D1208A15F7018A111B2190
:101610008A157808A400201220088316870000008D
:101620008312A0152008831687008312871D162BAE
:1016300000001A2B000020162008831687000000E7
:101640008312201620088316870000008312A0153D
:10165000200883168700000083120712201220083A
:1016600083168700000083128711A01120088316BB
:101670008700AA308312BB008A11D1208A150A3054
:10168000BB008A11D1208A152012200883168700FA
:1016900000008312A0152008831687008312871D7F
:1016A0004F2B0000532B00002016200883168700C4
:1016B0000000831220162008831687000000831282
:1016C000A01520088316870000008312071220123D
:1016D000200883168700000083128711A0112008BC
:1016E00083168700AB308312BB008A11D1208A1584
:1016F000F7018A111B218A157808A50020122008FD
:101700008316870000008312A01520088316870027
:101710008312871D892B00008D2B000020162008C6
:101720008316870000008312201620088316870086
:1017300000008312A0152008831687000000831282
:1017400007122012200883168700000083128711D9
:10175000A011200883168700AA308312BB008A11CB
:10176000D1208A150B30BB008A11D1208A15201296
:1017700020088316870000008312A0152008831616
:1017800087008312871DC22B0000C62B0000201685
:101790002008831687000000831220162008831675
:1017A000870000008312A015200883168700000020
:1017B000831207122012200883168700000083126C
:1017C0008711A011200883168700AB308312BB005D
:1017D0008A11D1208A15F7018A111B218A157808F0
:1017E000A600201220088316870000008312A0158F
:1017F0002008831687008312871DFC2B0000002C15
:10180000000020162008831687000000831220168F
:1018100020088316870000008312A0152008831675
:101820008700000083120712201220088316870009
:10183000000083128711A011200883168700AA30A8
:101840008312BB008A11D1208A150430BB008A1193
:10185000D1208A15201220088316870000008312E9
:10186000A0152008831687008312871D352C0000E1
:10187000392C0000201620088316870000008312F0
:10188000201620088316870000008312A015200868
:101890008316870000008312071220122008831687
:1018A0008700000083128711A0112008831687008B
:1018B000AB308312BB008A11D1208A15F7018A113F
:1018C0001B218A157808A70020122008831687009C
:1018D00000008312A0152008831687008312871D3D
:1018E0006F2C0000732C0000201620088316870040
:1018F0000000831220162008831687000000831240
:10190000A0152008831687000000831207122012FA
:10191000200883168700000083128711A011200879
:1019200083168700AA308312BB008A11D1208A1542
:101930000530BB008A11D1208A1520122008831699
:10194000870000008312A0152008831687008312E9
:10195000871DA82C0000AC2C000020162008831640
:1019600087000000831220162008831687000000DD
:101970008312A01520088316870000008312071227
:101980002012200883168700000083128711A011FF
:10199000200883168700AB308312BB008A11D12048
:1019A0008A15F7018A111B218A157808A8002012D0
:1019B00020088316870000008312A01520088316D4
:1019C00087008312871DE22C0000E62C0000201601
:1019D0002008831687000000831220162008831633
:1019E000870000008312A0152008831687000000DE
:1019F000831207122012200883168700000083122A
:101A00008711A011200883168700AA308312BB001B
:101A10008A11D1208A150630BB008A11D1208A157F
:101A2000201220088316870000008312A0152008CA
:101A3000831687008312871D1B2D00001F2D0000B9
:101A40002016200883168700000083122016200825
:101A50008316870000008312A015200883168700D4
:101A6000000083120712201220088316870000004E
:101A700083128711A011200883168700AB308312D0
:101A8000BB008A11D1208A15F7018A111B218A1502
:101A90007808A9002012200883168700000083120E
:101AA000A0152008831687008312871D552D00007E
:101AB000592D00002016200883168700000083128D
:101AC000201620088316870000008312A015200826
:101AD0008316870000008312071220122008831645
:101AE0008700000083128711A01120088316870049
:101AF000AA308312BB008A11D1208A150730BB009F
:101B00008A11D1208A152012200883168700000030
:101B10008312A0152008831687008312871D8E2D3F
:101B20000000922D00002016200883168700000078
:101B30008312201620088316870000008312A01548
:101B40002008831687000000831207122012200845
:101B500083168700000083128711A01120088316C6
:101B60008700AB308312BB008A11D1208A15F701A0
:101B70008A111B218A157808AA00201220088316D2
:101B8000870000008312A0152008831687008312A7
:101B9000871DC82D0000CC2D0000201620088316BC
:101BA000870000008312201620088316870000009B
:101BB0008312A015200883168700000083120712E5
:101BC0002012200883168700000083128711A011BD
:101BD000200883168700AA308312BB008A11D12007
:101BE0008A150230BB008A11D1208A1520122008E4
:101BF0008316870000008312A01520088316870033
:101C00008312871D012E0000052E000020162008DB
:101C10008316870000008312201620088316870091
:101C200000008312A015200883168700000083128D
:101C300007122012200883168700000083128711E4
:101C4000A011200883168700AB308312BB008A11D5
:101C5000D1208A15F7018A111B218A157808AB005B
:101C6000201220088316870000008312A015200888
:101C7000831687008312871D3B2E00003F2E000035
:101C800020162008831687000000831220162008E3
:101C90008316870000008312A01520088316870092
:101CA000000083120712201220088316870000000C
:101CB00083128711A011200883168700AA3083128F
:101CC000BB008A11D1208A150330BB008A11D120B4
:101CD0008A15201220088316870000008312A015A1
:101CE0002008831687008312871D742E0000782E2B
:101CF000000020162008831687000000831220169B
:101D000020088316870000008312A0152008831680
:101D10008700000083120712201220088316870014
:101D2000000083128711A011200883168700AB30B2
:101D30008312BB008A11D1208A15F7018A111B2159
:101D40008A157808AC00201220088316870000004E
:101D50008312A0152008831687008312871DAE2EDC
:101D60000000B22E00002016200883168700000015
:101D70008312BC012208BB00BC00BB0121083B0749
:101D8000AD003C08AE000318AE0A2E08BC002D08BA
:101D9000BB00BE010A30BD008A11E6298A15790808
:101DA000BC007808BB0011303B02AD003C08AE001F
:101DB0000130031C0230AE02BC012408BB00BC0091
:101DC000BB0123083B07AF003C08B0000318B00A72
:101DD000BC012608BB00BC00BB0125083B07B100C5
:101DE0003C08B2000318B20ABC012808BB00BC00C2
:101DF000BB0127083B07B3003C08B4000318B40A32
:101E0000BC012A08BB00BC00BB0129083B07B50088
:101E10003C08B6000318B60ABC012C08BB00BC0085
:101E2000BB012B083B07B7003C08B8000318B80AF1
:101E30001B3003178D0000308F0003101330031385
:101E4000BB008A1174218A15103084002E08BC0052
:101E50002D08BB008A110D228A15263003178D002C
:101E600000308F00031004300313BB008A1174216B
:101E70008A15293003178D0000308F0003100F30B2
:101E80000313BB008A1174218A15103084003008B6
:101E9000BC002F08BB008A110D228A1532300317AF
:101EA0008D0000308F00031006300313BB008A1131
:101EB00074218A15363003178D0000308F0003100F
:101EC00007300313BB008A1174218A151030840077
:101ED0003208BC003108BB008A110D228A153B3044
:101EE00003178D0000308F00031006300313BB0072
:101EF0008A1174218A153F3003178D0000308F003E
:101F0000031011300313BB008A1174218A1510309D
:101F100084003408BC003308BB008A110D228A15E6
:101F2000493003178D0000308F0003100630031373
:101F3000BB008A1174218A154D3003178D000030C3
:101F40008F0003100E300313BB008A1174218A1511
:101F5000103084003608BC003508BB008A110D2201
:101F60008A15553003178D0000308F00031406309A
:101F70000313BB008A1174218A15593003178D0091
:101F800000308F00031006300313BB008A11742148
:101F90008A15103084003808BC003708BB008A114D
:101FA0000D228A155D3003178D0000308F00031459
:101FB0000D300313BB008A1174218A150830BB0051
:101FC000FA30BC008A1160218A15BB0BE02F6E2805
:021FD0006300AC
:04400E00F52CFF3F4F
:00000001FF
